:020000040800F2
:10000000D80E0020615F00088D5D00088F5D00083C
:10001000915D0008935D0008955D0008795F000818
:10002000000000000000000000000000975D0008D4
:10003000995D0008000000009B5D00089D5D0008C0
:100040007D5F0008815F0008855F0008895F000808
:100050008D5F0008915F0008955F0008995F0008B8
:100060009D5F0008A15F0008A55F0008A95F000868
:10007000AD5F0008B15F0008B55F0008B95F000818
:10008000BD5F0008C15F0008C55F0008C95F0008C8
:10009000CD5F0008D15F0008D55F0008D95F000878
:1000A000DD5F0008E15F0008E55F0008E95F000828
:1000B000ED5F0008F15F0008F55F0008F95F0008D8
:1000C000FD5F000801600008056000080960000885
:1000D0000D60000811600008156000081960000834
:1000E0001D600008216000082560000829600008E4
:1000F0002D60000831600008A15D0008356000082F
:10010000396000083D600008416000084560000853
:1001100049600008000000004D60000851600008C0
:100120000000000055600008596000085D6000088C
:100130006160000865600008696000086D60000883
:100140007160000875600008796000087D60000833
:10015000BD5D0008816000088560000840F0200057
:1001600070472DE9F14FB0B0924604910DF1420174
:100170003A9A2B9199464A7000200AE01AF8011B1E
:100180000498309A90470028049000F041860D981A
:10019000401C0D909AF8000050B12528EED10021A6
:1001A00000220791089209910A920B910C9204E0A7
:1001B0000D9800F02FBE41F001011AF8010F202820
:1001C000F9D023280CD02B2804D02D2805D0302896
:1001D00009D00BE041F00201EFE741F00401ECE748
:1001E00041F00801E9E741F01001E6E72A280FD1C4
:1001F000D9F8002052F8040BC9F8002000280F900D
:1002000003D540420F9041F004010AF1010A14E0C5
:100210000F92DFF8083C0AE00F98984205DA00EBED
:10022000800402EB4402303A0F920AF1010A9AF874
:100230000020A2F130000A28EED39AF800002E2800
:1002400003D04FF0FF320E9229E01AF8010F2A284E
:1002500009D1D9F8000050F8042BC9F800000E921B
:100260000AF1010A1BE02D280CBF0AF1010A002047
:1002700000220E92DFF8A44B0BE040B90E9AA24286
:1002800005DA02EB820503EB4503303B0E930AF1DE
:10029000010A9AF80030A3F130020A2AEDD3ADF832
:1002A00040100FF67C309AF8001000F0FBFE08B109
:1002B0001AF8010B8DF842009DF84200682805D11C
:1002C0009AF8000068280CD1622106E06C2804BF6F
:1002D0009AF800006C2804D171218DF842100AF1BF
:1002E000010A12A806901AF801BBBBF125012CD017
:1002F0001C3900F09481091F022940F290811339C2
:1003000000F0B884093900F08A81891E00F04D851B
:10031000491E00F0FA84491E022940F28081091F1B
:1003200000F0F384491F00F0EF80491E00F0A28422
:10033000491E00F0D780C91E0CD0891E00F09A8497
:10034000C91E00F0978400F03BBD012307932521CF
:1003500000F033BDD9F8000050F8044BC9F8000094
:10036000002C059440F0AB802B994878002800F0D1
:10037000A1804FF0FF340FF6B02000F09FFE241A4A
:1003800040F0468500F028BD01236A4602A93046A8
:1003900000F00EFE002840F03B85641EF4D130963C
:1003A000079C12AF74B1309E17F8011B0498B04738
:1003B0000028049000F02C850D98401C641E0D90C0
:1003C000F2D130960A9C3021002C8DF800100CDD03
:1003D000309E01236A4602A9304600F0E9FD00285C
:1003E00040F01685641EF4D13096059F089C74B1C8
:1003F000309E17F8011B0498B0470028049000F0C5
:1004000007850D98401C641E0D90F2D130960B9C10
:100410003021002C8DF800100CDD309E01236A463F
:1004200002A9304600F0C4FD002840F0F184641EAB
:10043000F4D1309605980899099C471874B1309EFC
:1004400017F8011B0498B0470028049000F0E084DE
:100450000D98401C641E0D90F2D130960C9C3021FA
:10046000002C8DF800100CDD309E01236A4602A995
:10047000304600F09DFD002840F0CA84641EF4D18F
:1004800030969DF8400041077FF584AE2020002D76
:100490008DF800007FF77EAE309C01236A4602A9EA
:1004A000204600F085FD002840F0B2846D1EF4D196
:1004B00030946FE60FF65830059000F08DBC0E9D1D
:1004C000002D04D5204600F019FE044607E02A4618
:1004D000204600F01DFE002814BF041B2C46089483
:1004E00000F07ABCD9F8001051F8040BC9F80010DC
:1004F00020F00004002121F0FF35CDE9024512ABC8
:100500000593782100F04DBC2B99487820B14FF02D
:10051000FF340FF6CC2030E79DF84200622860D00F
:10052000682817D06A283FD06C2806D0712847D099
:1005300074282CD07A281DD062E0D9F8001051F828
:10054000040BC9F80010002866D14FF0FF340FF6F5
:10055000A82012E7D9F8001051F8040BC9F80010D0
:1005600020B94FF0FF340FF6902006E70D99018077
:1005700000F032BCD9F8001051F8040BC9F8001093
:10058000002849D14FF0FF340FF66C20F5E6D9F87A
:10059000001051F8040BC9F8001000283CD14FF0AE
:1005A000FF340FF65420E8E6D9F8001051F8040B98
:1005B000C9F8001080B94FF0FF340FF63C20DCE69C
:1005C000D9F8001051F8040BC9F8001020B94FF009
:1005D000FF340FF62420D0E60D9AD317C0E900238C
:1005E000FAE3D9F8001051F8040BC9F8001020B94B
:1005F0004FF0FF340FF60020BFE60D990170EBE3DA
:10060000D9F8001051F8040BC9F8001020B94FF0C8
:10061000FF340FF6E410B0E60D990160DCE39DF8BD
:1006200042004C2807BFD9F80010CA1DD9F80000B5
:10063000C21D22F00702C9F80020D2E900010832E9
:10064000C9F80020CDE90201C80F02D007982D217A
:100650000AE0BDF84000810702D507982B2103E08E
:10066000C00705D50798202112AA1154401C0790F5
:1006700012A807994BF0200300EB010CDDE9020101
:10068000CDE92C01612BCDF814C021AC0BD00E9814
:10069000002848BF062105D404BF4BF0200067287E
:1006A00001D101210E91DDE902014F0047EAD07727
:1006B0007E15FF174FF0FF32974208BF964210D1C8
:1006C000090341EA10510003002908BF002808D09F
:1006D000ABF1610503211A2D089118D30FF63811DB
:1006E00010E0DDE902014A00521512F1010F11D1AB
:1006F00008030FD1ABF1610503211A2D08911FD317
:100700000FF61C110322604600F02EFD64E30FF685
:100710000411F7E7DDE902016A4600F031FDCDE999
:1007200002014BF02000612811D1059830210170A1
:10073000821C0592BBF1610F0CBF7821582102E0A9
:100740000FF6D801DEE741700798801C0790DDE9BD
:10075000020120F0000231F0004308BF002A02D15C
:100760000026002542E14BF02008B8F1610F40F06F
:1007700092800E98002847BF21210191401C0190D2
:10078000019FDDE92C017F1C00220023DDE90245E9
:1007900000F02EFD38BF85F0004500998DF88420CB
:1007A000091F002F00910DF1850632DD20462946F4
:1007B0000022002300F036FD2BD21C2200F04CFD5D
:1007C00004460D4600F0E6FDFF1F002F804609DDC0
:1007D00000F0FCFD02460B462046294600F0BEFE16
:1007E00004460D46F01D0721B8F1000F0CDD491E2F
:1007F0005EBF08F00F0200F8012D4FEA2818F3D56C
:1008000002E0002200F8012D491EFAD5C61D002F76
:10081000CCDC0DF18500361A01980DF18504864275
:10082000D8BF304600282FD4B04206DA0DF185013A
:100830000A5C082AA8BF0F2100DA0021024621AB7A
:10084000134400E0401E13F80159521E8D42F9D0A6
:100850000F2904D10DF185018B5C5B1C8B54002AA0
:1008600004D50099091D21AC401C0091411E0BD4F8
:10087000621813783033DDB23A2DA4BF5B443A3BA3
:10088000491E02F80139F4D50E99002940F1AC80D7
:10089000421E0E92A8E00099DFF8042747F2975015
:1008A000414391FBF2F20092DDE92C45C2F10702CF
:1008B000002A25F0004504DD2046294600F04CFBC7
:1008C0000BE052420020DFF8DC1600F045FB024648
:1008D0000B462046294600F0B3FE04460D46B8F10B
:1008E000660F06BF009F0A3706270E983F18142F81
:1008F000C8BF142730208DF884000DF18506002F25
:1009000034DD2046294600F0BFFF01460A4606F1C5
:10091000080304200A26B2FBF6F606EB860EA2EBCD
:100920004E02303203F8012C0A22B6FBF2F202EB3F
:10093000820EA6EB4E063036401E03F8026DE9D15A
:10094000083F002F03F10806D9DD084600F0AEFF8E
:1009500002460B462046294600F000FE0022DFF842
:10096000483600F0B1FF04460D46CAE70DF1850098
:10097000361A0DF1850404E00098401E761E0090A2
:10098000641C20783028F7D0B8F1660F02D10098A7
:10099000401C04E0B8F1650F0CBF012000200E9947
:1009A00040188642B8BF701E00281DD4B04204DA39
:1009B000215C3429C8BF392100DC30210246631E86
:1009C0009D1800E0401E15F80169521E8E42F9D0B4
:1009D000392902D1A15C491CA154002A04D50099EF
:1009E000491C1C46401C00910646009D01F05AF827
:1009F000406A0778DDF8388030B2002802DC012632
:100A00000FF220644BF02000662808BF6D1C16D042
:100A1000672845D128B210F1040F47DB404545DA7D
:100A20009DF840006D1C010703D430B24045D8BF8B
:100A3000804628B2B8EB000848BF4FF000080FFA14
:100A400085FBBBF1000F00F3B4800898411C0891AE
:100A5000302205990A54B8F1000F03DC9DF84000DC
:100A6000010704D50898411C089105990F5418EB0B
:100A70000B0FB8BFC8F100052DB26842454432B231
:100A80000B909542B8BF2E46059B089836B2099642
:100A900032462146184400F067FBAD1B0C95D2E0AE
:100AA000BBF1610F17D14FF0700B19E030B2404528
:100AB00004DA9DF840100A0758BF8046B8F10108D3
:100AC00048BF4FF00008BBF1670F14BF4FF0450B54
:100AD0004FF0650B04E0BBF1410F08BF4FF0500B26
:100AE0000898411C0891B8F1000F059914F8012BE2
:100AF0000A5403DC9DF8400001071AD50898411CF0
:100B00000891B8F1000F05990F5412DD761E30B22E
:100B10008045B8BF46460598089B32B22146184426
:100B200000F022FB089936B271180891A8EB060074
:100B30000B9005980899084429B2002980F800B064
:100B400003D42B224270821C04E02D2242700D46F9
:100B5000821C6D4200212CAB28460AE004460A2084
:100B600094FBF0F000EB8005A4EB450403F8014B87
:100B7000491C00B20028F1DC012906DC4BF0200002
:100B8000652804BF302002F8010B00292CAB08D1E6
:100B9000302002F8010B06E0491E585C303002F8A4
:100BA000010B0029F8DC059908980844121A0992EB
:100BB00049E030B229B288421CDA0598089B32B26B
:100BC0002146184400F0D0FA089936B271180891FD
:100BD000ABEB0600B8F1000F0B9003DC9DF8400072
:100BE000020704D5059847540999491C0991CDF885
:100BF000308028E00598089B2AB22146184400F06E
:100C0000B3FA0898761B5844B8F1000F089003DC3B
:100C10009DF840100A0703D5411C089105990F540F
:100C200030B28045B8BF46460598089B32B204EB07
:100C30000B01184400F098FA089836B23018089062
:100C4000A8EB06000B909DF8400000F0140010285F
:100C500040F0C280079A08980B99821809988A1860
:100C600082180C980F998018884280F2B580081A73
:100C70000A90B1E09DF84200622808D068280ED0A2
:100C80006A2814D06C281FD0712810D01CE0D9F825
:100C9000001051F8040BC9F80010C0B21AE0D9F8DE
:100CA000001051F8040BC9F8001080B212E0D9F816
:100CB0000000C21D22F00702C9F80020D2E900019D
:100CC0000832C9F8002006E0D9F8001051F8040BEA
:100CD000C9F800100021CDE902019DF8400001078C
:100CE0005AD5DDE90223002B08BF002A54D04BF06F
:100CF0002000782850D1079812A930220A54401CAD
:100D0000431C079301F800B046E09DF842006228BA
:100D100008D068280ED06A2814D06C281FD07128FB
:100D200010D01CE0D9F8001051F8040BC9F80010DD
:100D300040B21AE0D9F8001051F8040BC9F80010BD
:100D400000B212E0D9F80000C21D22F00702C9F873
:100D50000020D2E900010832C9F8002006E0D9F8E5
:100D6000001051F8040BC9F80010C117CDE90201B9
:100D7000002902D507982D210AE0BDF8400081071F
:100D800002D507982B2103E0C00705D5079820213D
:100D900012AA1154401C079012A80799014405910A
:100DA000594602A800F04EF816E001200790D9F845
:100DB000000050F8041BC9F800008DF848100BE043
:100DC00001212522BBF1000F07918DF8482003D0A7
:100DD000022207928DF849B00F9D07990A986D1A63
:100DE00008992D1A0B986D1A09992D1A0C986D1ADD
:100DF0009DF840102D1A48073FF5D2AA2021002D5A
:100E00008DF800107FF7CCAA309E2C46FFF7BCBAB5
:100E10004FF0FF3031B0BDE8F08F0000CBCCCC0CF0
:100E2000686A6C747A4C00007072696E74665F73E5
:100E30003A2062616420257320617267756D656E6A
:100E4000740000002DE9FC4707468A463C6950467D
:100E50006F2808BF082505D0FFF780F9782814BF50
:100E60000A251025D7E900013C2680468946BAF1BB
:100E7000640F18BFBAF1690F05D1002903D5D8F165
:100E8000000869EB4909B9F1000F08BFB8F1000F7C
:100E90000CD1386B50B9082D3AD197F838000107BA
:100EA00036D530223B2684F83B2031E08DF800A077
:100EB000404649462A46EB1700F0FAFD3032D0B2E0
:100EC000761E3A2801960EDAA255404649462A4631
:100ED000EB1700F0EDFD80465FEA010908BFB8F1AD
:100EE000000F05D108E09DF800001218513AEBE719
:100EF000F868A1198842DBD3082D09D197F838008A
:100F0000010705D5A05D302802D0761E3020A055FF
:100F1000C6F13C03BB61A119F960386B834208DA62
:100F2000C31A3B624FF6EF70398F01403987BDE835
:100F3000F38700280ED597F8380000F01400102829
:100F400008D17A6B7969386A521A121AD21A002AB1
:100F5000C8BF3A62BDE8F3872DE9D04306460F4685
:100F600014464FF00008DFF8449012E0E00707D580
:100F700042464B463046394600F0A6FC06460F4630
:100F80004046494642464B4600F09EFC641080466F
:100F90008946002CEAD130463946BDE8D0830000AE
:100FA000A08601000000F03F84D797410000244054
:100FB000F8B505460E4617461C4600205CB117F8EA
:100FC000011BB068A847B06030B1F06A401CF06205
:100FD0000020641EF3D1F2BD4FF0FF30F2BD0000DF
:100FE0007072696E74665F733A20256E206469734F
:100FF000616C6C6F776564007072696E74663A201C
:1010000062616420256E20617267756D656E740083
:10101000000000006E616E004E414E00696E660079
:10102000494E46003000F0B4024610689568131827
:10103000506803EB5004C00748BF4D44A3422DD075
:1010400013F8016B16F0030004BF13F8010BC01C6A
:1010500031090F2907D113F8011B0F3103E013F8F1
:10106000017B05F8017B401EF9D10029E6D013F879
:10107000010BC6F38106032E08BF13F8016B00EBCA
:101080000620404228440026B71E8F421EBF10F89B
:10109000017B05F8017B761CF6D1CFE7F0BC02F1AD
:1010A0000C007047C9B202788A421AB11CBF10F80E
:1010B000012FF9E718BF002070472E0080B500B956
:1010C00006A005490B681BB122220021984701E0C8
:1010D00000F071FD222002BDD40A0020636F6E7300
:1010E000747261696E742068616E646C65723A2016
:1010F000626164206D6573736167650000F10103CF
:1011000010F8011B11B110F8011BFBE7C01A704762
:10111000C9B2830706D0521E22D310F8013B994270
:10112000F7D11FE0083A13D302F1040241EA01218A
:1011300041EA014150F8043B121F21BF4B40A3F18B
:10114000013C2CEA030C1CF0803FF3D0C9B2001F15
:10115000083210F8013B521E28BF91EA030FF8D85D
:1011600018BF0120401E70474AB1000011F8013B32
:10117000521E00F8013B1CBF11F8013BF8E7704715
:1011800010B5144600F002F8226010BDC1F30A53F6
:1011900043B14A0012F5001F28D2A3F2FE32A1EBA0
:1011A0000251704750EA410C20D001F0004C31EA66
:1011B0000C01B1FA81F204BFB0FA80F3D2180B3AF5
:1011C000B2F120032CBF00FA03F1914041EA0C0177
:1011D0003EBFC2F1200C20FA0CF31943904052425A
:1011E00040F2FD33D21A01EB0351704700227047E1
:1011F00041EA030C50EA4C0C52EA0C0C4FF4001C70
:1012000009D307D01CEB410F9CBF1CEB430F8B4253
:1012100008BF824270471CEB430FFBD8994208BFBE
:101220009042704741EA030C50EA4C0C52EA0C0C15
:101230004FF4001C09D307D01CEB410F9CBF1CEBE3
:10124000430F994208BF904270471CEB410FFBD8F7
:101250008B4208BF82427047124254D440F2FF7C56
:101260001CEA11530FD0634531D09B1863453CBF36
:1012700001EB0251704701F0004141EA0C5100209E
:10128000AFF30080704750EA410320D001F0004CDA
:1012900091EA0C011CD0B1FA81F30B3B9A420DD9B3
:1012A000D21A994051EA0C01C3F1200C20FA0CFC2F
:1012B00061449840531C40F2FF7CD7E7914041EADB
:1012C0000C01C2F1200C20FA0CF319439040704736
:1012D000B0FA80F31533202BE0D3202AEED3203A46
:1012E000203B9A4209D9D21A00FA03F141EA0C01D3
:1012F0000020531C40F2FF7CB8E700FA02F141EAFB
:101300000C0100207047524240F2FF7C1CEA11534E
:101310000DD06345DBD0B2EB030C3CBFA1EB025117
:1013200070470CF1010221EA035141F4801150EAA7
:10133000410CCCD001F0004C352A27DC30B481EAD6
:101340000C01B2F1200309DAC2F12003044601FACC
:1013500003F5D0402843D1409C400CE0C3F120026B
:10136000450020FA03F418BF44F0010421FA03F009
:1013700091400C43002174F1004550F1000051EB05
:101380000C01244230BC7FF47BAF704761460020E3
:1013900076E74300C1F30A5340F21E42D31A0CDD34
:1013A000CA0283F3070342EA505242F00042DA4095
:1013B00002EBE17282EAE17070476FEAE17203F2D8
:1013C000E13008B182F000407047000010F00041A9
:1013D00060B148BF4042B0FA80F29040D21CC2F5E2
:1013E000846241EA025202EBD021400570470000BE
:1013F000841A71EB030604D26E40001BB14112192E
:1014000073414FF4001C1CEB410F34BF7CEB4306CF
:1014100083E00C0DA4EB1356362E00F37C80012ED6
:1014200045EAC32341DC43EA525312BFD20292027F
:101430005B08240545EAC12141EA5051D2EBC020A6
:10144000994125D407D1B0FA80F610FA06F162D09E
:101450000020203608E0B1FA81F6B140C6F1200242
:1014600020FA02F21143B0404FEAF474B4EB465450
:1014700034F001064FEA74040AD8D6F50016760D4A
:1014800004F00044F04061FA06F25040F140484058
:10149000C00A40EA415021F0004128BF5FEA5005F0
:1014A00050F1000044EBD12135E0DB0A45EAC121CF
:1014B000C90AB6F120050EDD42EA0242120CC5F15E
:1014C000200603FA06F6EB4042EA06056D42984113
:1014D00061F100010DE062FA06F5F240554063FA51
:1014E00006FC82EA0C02F3405A406D42904161EBE7
:1014F000030111F4801F05D1641E620502D06D0046
:101500004041494121F48011430875F1004350F1F5
:10151000000041EB045170BC70471CEB410F15D229
:1015200023F0004352EA43060BD04FEA4C0CBCEBCD
:10153000410F04D80C0D661E342EB7DDEBE7801A80
:10154000994150EA410608BF0021E4E708BF1CEBBF
:10155000430F28BF6FF00001DDE7000070B491EA8F
:10156000030F4FF000457FF543AF6B40841A71EBDA
:10157000030603D2001BB141121973414FF4001C42
:101580001CEB410F34BF7CEB430442E00C0DA4EB99
:101590001356352E4FDC45EAC323DB0A45EAC12149
:1015A000C912B6F120050DDD63FA05F6EB4086EAB7
:1015B0000305124218BF45F00105C01851F10001A2
:1015C0000CD213E062FA06F5F2405540F3415A405E
:1015D000B340F3405A408018594107D349085FEAA5
:1015E00030005FEA350528BF45F0010501F580119F
:1015F000420875F1004250F1000041EB04514E00E9
:1016000016F5001F70BC38BF70470020090D090592
:1016100070471CEB410F10D252EA43060BD0BCEBD3
:10162000410F05D80C0DAB43661E342EB6DD02E02B
:10163000AB438018594170BC704770BC70470000C4
:10164000F0B540F2FF7581EA030C0CF0004C15EA8E
:1016500011541DBF15EA1357AC42AF42E5E0BC413F
:10166000C1F31301C3F31303801A994143F48013A8
:1016700004D2641E0018494180185941C90241EA48
:101680005051B1FBF3F603FB1611A2FB0675D7EB25
:10169000C020A94102D2761E80185941C90241EAF0
:1016A0005051B1FBF3FE03FB1E11A2FB0E75D7EBED
:1016B000C020A94103D2AEF1010E80185941890220
:1016C00041EA9051760546EA8E2EB1FBF3F603FB14
:1016D0001611A2FB0675D7EB8020A94102D2761E17
:1016E00080185941C90241EA50514EEA060EB1FB39
:1016F000F3F603FB1611A2FB0675D7EBC020A94138
:1017000002D2761E80185941C90241EA5051B1FBFC
:10171000F3F703FB1711A2FB0735D3EBC020A94158
:1017200067F100070CBF004247F0010766F3D527B9
:101730004FEA1E31B80814F5806412DDBD0775F15B
:10174000004250EB0E5051EB045111F5801F5CBF6D
:1017500041EA0C01F0BD4CF07F6141F0E041002016
:10176000F0BDBD076D0840EA0E5041F48011D4F180
:101770000104B4F120060ADAC4F120060200E040B8
:1017800001FA06F3E1401843B24015430EE0342C51
:1017900013DCC6F1200445EA40056D0820FA06F284
:1017A000154321FA06F0A1400D43002175F10042D6
:1017B00050F1000051EB0C01F0BD00205FEA0C017C
:1017C000F0BDCFB992185B41B3FA83F704BFB2FA08
:1017D00082F6BF190B3FB7F120062FBF02FA06F3BE
:1017E000BB40C7F1200622FA06F638BF3343BA40A1
:1017F0001CB1E419641E33E77F4231F00041B1FAB5
:1018000081F404BFB0FA80F6A4190B3CB4F12006B1
:101810002FBF00FA06F1A140C4F1200620FA06F617
:1018200038BF3143A0403C1B1AE7AC421ABF05EA5F
:101830001357AF4212E050EA41061CBF52EA43067A
:10184000BFE750EA4107304661461CBF41EA0551F7
:10185000F0BD52EA430C08BFC143F0BD00204FF475
:10186000001616EB410F98BF16EB430F08BF16EB9F
:10187000410F24BFC14305E016EB430F0CBF614687
:101880004CEA0551F0BD0000400D40F21E4C40EA0C
:10189000C120BCEB115C40F0004003D48CF3070185
:1018A000C84070476FEAE1707047000050B1B0FA6D
:1018B00080F18840C91CC1F58461090501EBD02184
:1018C000400570470146704730B540F2FF7C1CEA86
:1018D00011541DBF1CEA1355644565453FE064196A
:1018E00081EA030C6FF35F530CF0004C43F4801358
:1018F000C90241F0004141EA505EC5021100A5FB5A
:10190000020200284FF00000EEFB01204FF0000122
:10191000E3FB052118BF42F00102401800214941B4
:10192000E3FB0E01A4F580640D0302D2921840413E
:10193000494154F1010470DD450872F1004250F153
:10194000000051EB0451A1F5801102D441EA0C01D1
:1019500030BD40F2FF7E4CEA0E51002030BD0CEA53
:101960001355644518BF654581EA030C0CF0004C23
:1019700041D050EA410E1CBF52EA430E02E06146DC
:10198000002030BD24422C441BD15FEA050EF6D066
:10199000090302BF01460020AEF1140EB1FA81F531
:1019A000AEEB050401FA05FE0C35C5F1200100FA85
:1019B00005F5C8404EEA000E6FF35F5343F4801301
:1019C0009CE733F00043B3FA83F504BFB2FA82FE1A
:1019D00075440B3D641BB5F1200E2FBF02FA0EF3C8
:1019E000AB40C5F1200E22FA0EFE38BF43EA0E03CB
:1019F000AA40641C7CE750EA410E14BF52EA430E31
:101A00006FF000014FF4001515EB430F8EBF194620
:101A100015EB410F9DE7B4D830BDD4F10104B4F10A
:101A200020050FDAC4F12005520828BF42F0010258
:101A300010FA05FE01FA05F57244E2BFE0402843C2
:101A4000E1400FE0352C9ADCC5F1200452EA400257
:101A500020FA05F218BF42F0010231FA05F0A14068
:101A60000A43002172F1004250F1000051EB0C01D9
:101A700030BD0000FFE741381A288041C00F704791
:101A8000A0F10901052901D3202801D101207047C7
:101A900000207047A0F141011A2938BF203070475B
:101AA000014870470148704748000020100000209E
:101AB000D3BBD9B1B2F5803F5BD2022A1ED98C4686
:101AC000B1FBF2F102FB11C31B0443EA1043B3FB69
:101AD000F2FC02FB1C3380B240EA0343B3FBF2F09A
:101AE00002FB103240EA0C4000237047022A05D95D
:101AF0008446B0FBF2F002FB10C270474AB105D138
:101B000000F0010249085FEA30007047002200231C
:101B1000704700F053B80B0002000021002070470E
:101B2000F7D3002200237047904271EB030CF2D3ED
:101B300070B5B1FA81F4B3FA83F52C1BA340C4F15C
:101B4000200532FA05F63343A2405FF00046E64036
:101B500002E05B085FEA3202841A71EB030524BFDE
:101B6000204629467641F4D302000B0030000021C4
:101B700070BD70B5B1FA81F4B2FA82F5C4F12004F7
:101B80006419B4F12006DAD3B2405FF00044F440A7
:101B9000002502E052085FEA3303C61A71EB020E19
:101BA00024BF3046714664416D41F3D302000B00FF
:101BB0002000290070BD012000F002B8704700002D
:101BC00080B5AFF30080024A11001820ABBEFBE7DE
:101BD0002600020038B5040001D1012032BD04F115
:101BE0008405686808B900F017F800F01AF808B121
:101BF00000F031F800F02CF8012804D000F004F8CF
:101C000021F02A0116E032BD2068416821F490419C
:101C1000416020688168704700212970204600F0EB
:101C20007FBF24206860206801684908490001607E
:101C3000A06A7047816000F004F8BDE8324000F00F
:101C4000AFBB2068016841F0010101602046704788
:101C5000204600F02DBA204600F03FBB38B5040006
:101C600001D1012032BD04F184052420686000F018
:101C700014F8226800200021106023685960216850
:101C80008860204600F0DDFF0020E86000216960E8
:101C9000A860E1662067297032BD206801684908A4
:101CA0004900016070472DE9F843054605F15406E7
:101CB000706B0C461746994620283ED10CB138006F
:101CC00001D101203AE00020F0632121716301F08D
:101CD00071F8378080467780A868B0F5805F04BFD0
:101CE000286900281ABF204600272746044611E02D
:101CF0000022802100F024F8D8B92868002C12BFF7
:101D000014F8011B37F8021BC1F3080181627088C7
:101D1000411E71807088CDF8009043460028E7D1BD
:101D20000022402100F00CF818B920207063002038
:101D300004E020207063032000E00220BDE8F2836D
:101D4000284600F074BB38B50346D3F88C00202831
:101D50000AD109B1100001D1012032BD00F006F80E
:101D6000BDE8384000F0ABBB022032BD0020D86691
:101D70001868DFF83843A0420CD04068040209D547
:101D8000186850E8004F054644F0806445E800407C
:101D90000028F5D1184670472868816848067047C2
:101DA0002DE9F04105462A68D36940F60F06104632
:101DB0000768D2F8088005F15C0407F0200003F002
:101DC000200133420ED1002914D018B95FEAC800AF
:101DD00040F18780A169002900F02F812846BDE8E5
:101DE000F0410847DFF838C818EA0C0F04BFDFF8E5
:101DF0003468374275D0DE0709D5FE0507D54FF0A8
:101E0000010EC2F820E0626B42F0010262639A07A1
:101E100048BF5FEAC87206D52E6802223262626B42
:101E200042F0040262635A0748BF5FEAC87206D5EF
:101E30002E6804223262626B42F0020262631A0769
:101E40000DD5002808BF18EA0C0F08D0D5F800C03F
:101E50000822CCF82020626B42F0080262631A0567
:101E600009D57B0107D52F684FF400623A62626B97
:101E700042F020026263626B002A31D039B110B99E
:101E80005FEAC80003D5A16909B128468847606B9D
:101E900029688A68510602D410F0280F1BD000F080
:101EA000D4F8FFF779FF11D500F0D2F8FCD1606AC1
:101EB00060B10FF2A171C166606A00F0BFFF002837
:101EC0000ED0606AC16EBDE8F04108472846BDE803
:101ED000F04100F0D4BF284600F0D1FF002060633D
:101EE000ABE02069012875D1D80673D5F90671D504
:101EF000102010622A6821889068420632D5626AF2
:101F00001068806C80B2002823D0884221DA60807B
:101F1000106D812816D000F0B4FCFCD100F0B8F8A8
:101F2000FCD100F0A8F8FCD1202020630021216121
:101F300000F09CF821F0100100F083F8F8D1606AFD
:101F400000F03EFF0220606121886088091A89B292
:101F500006E0884204BF106D81286ED102226261C2
:101F6000284633E062886088891A00281CBF88B23E
:101F7000002862D02A46106850E8003F054623F446
:101F8000907345E800300028F5D1106800F108038F
:101F900053E8003F00F10808DFF82C03034048E84D
:101FA00000300028F1D12020206300232361A361A9
:101FB000136853E8003F156823F0100345E800302C
:101FC0000028F5D10220606189B21046BDE8F041D9
:101FD00000F056BF18060AD5390658BF5FEA082038
:101FE00005D5E16949B32846BDE8F04108475806E0
:101FF00011D579060FD500F039F821F0400100F035
:1020000020F8F8D12020E0620021E1612846BDE8F7
:10201000F04100F036BF180206D5790004D52846F5
:10202000BDE8F04100F02EBFD80148BF002F04D515
:102030002846BDE8F04100F026BFBDE8F08141F43C
:10204000807142E8001000287047284600F0BDBAB1
:10205000296801F1080252E8001F286800F108030E
:1020600021F0400143E8001000287047286850E83C
:10207000001F02467047286800F1080151E8001F60
:1020800000F1080321F0400143E8001000287047E8
:10209000286800F1080151E8001F00F10803490811
:1020A000490043E800100028704700000024004663
:1020B000F8B504462268DFF8F40600251368A16825
:1020C000034020690B4361690343E0690B43034309
:1020D00013605168E06821F4405101435160DFF81A
:1020E0008417A3698A421CBF206A03439668DFF8FD
:1020F0007807DFF878E7064033439360D36A606A75
:102100000FF25C561B0940EA0313DFF86407DFF89F
:102110006477D3624FF4004372453AD13F6807F0C9
:102120000307032F5AD8DFE807F0025350564FF049
:10213000010CE1694FF6F077B1F5004F40F0908067
:10214000BCF1000F0FD0BCF1010F00F08180BCF199
:10215000040F0CD0BCF1080F00F07D80BCF1100F13
:1021600000F07C80A5E001F0B1F9002810D000F06B
:10217000ADF84A0802EB4002B2FBF1F0A0F1100109
:10218000B942EFD20740C0F3420007432068C7605E
:1021900090E0DFF8A4C762450CD13F6817F00C0748
:1021A00006D0042F14D0082F0FD00C2F13D015E019
:1021B000AC46BEE78A4211D1BF6807F00307032F80
:1021C0000CD8DFE807F01C0502084FF0040C07E00C
:1021D0004FF0080C04E04FF0100C01E04FF0200C21
:1021E0008A42A6D1BCF1020F09D0BCF1040F0AD07B
:1021F000BCF1080F15D0BCF1100F15D059E001F05B
:1022000073F9002856D0616A36F81120B0FBF2F657
:10221000626802EB42018E424BD31303B34205D2F4
:1022200047E001F034F9ECE71846ECE750080021EC
:1022300010EB0620DFF8A87751EB16610023FFF7BB
:1022400037FCA0F54076BE4233D22168C86031E049
:1022500001F041F989E701F01AF986E7184686E7A7
:10226000BCF1000F0CD0BCF1010F1AD0BCF1040F6F
:1022700009D0BCF1080F17D0BCF1100F17D018E02F
:1022800001F024F9B0B100F021F800EB5100B0FBEF
:10229000F1F0A0F11001B9420BD2226880B2D060F7
:1022A00008E001F018F9EDE701F0F1F8EAE7184667
:1022B000E9E7012504F16800012100234180018044
:1022C000C36003612846F2BDFEFFFFEF626A6168EA
:1022D00036F81230B0FBF3F0704790F828100A0778
:1022E00006D502685368816B23F400430B435360A7
:1022F00090F82810CA0706D502685368C16A23F40B
:1023000000330B43536090F828108A0706D5026803
:102310005368016B23F480330B43536090F828100B
:102320004A0706D502685368416B23F480230B43A8
:10233000536090F82810CA0606D502689368C16BEE
:1023400023F480530B43936090F828108A0606D537
:1023500002689368016C23F400530B43936090F878
:1023600028104A0610D502685368416C23F4801384
:102370000B435360436CB3F5801F05D15368816CE8
:1023800023F4C0030B43536090F828100A0606D5C7
:1023900001684A68C06C22F4002202434A60704718
:1023A000F8B5054605F184040020E06000F002FD68
:1023B000064628686FF07E4701680A0711D5009726
:1023C000334600224FF40011FFF7BAFC48B1FFF783
:1023D0004DFE21F08001FFF734FEF8D1202060602F
:1023E00017E0286801684A0717D50097334600228E
:1023F0004FF48001FFF7A4FC78B1FFF737FE21F41A
:102400009071FFF71EFEF8D1FFF742FEFCD12020AD
:10241000A060002121700320F2BD202060602021F7
:10242000A1600020E866002129672070F2BD2DE937
:10243000F04105460E4690461F46069C2868C16935
:102440003140B1420CBF01200020404535D114F18C
:10245000010FF3D000F0AEFCC01B844200D314B9CE
:102460000320BDE8F081286801684A07E6D5802E80
:1024700018BF402EE2D0C169080704D42968C86992
:102480000105DBD50CE02A6808201062FFF7DDFDAE
:1024900005F184000821C160002202700120E0E7FC
:1024A00029684FF400600862FFF7CFFD05F1840052
:1024B0002021C16000220270D2E70020D1E750B590
:1024C0000346996503F15C010A804A800020886117
:1024D0009868FF24B0F5805F04D1186990B940F284
:1024E000FF140FE018B9186960B17F2007E0B0F160
:1024F000805F06D1186908B97F2403E03F208880F7
:1025000001E000248C800020486322240C631868BA
:1025100000F098F844F0010446E800400028F6D1A5
:102520008868B0F1005F21D1888982421ED39A6801
:10253000B2F5805F04BF1869002803D10FF2593249
:102540008A6109E00FF27D248C61186920B100F0E6
:102550002FF8FFF774FDFAD100F02FF841F0805109
:1025600044E800100028F7D1002050BD9868B0F56D
:10257000805F04BF186900280CD10FF24D128A61E8
:10258000186850E8001F024641F02001FFF759FD8E
:10259000F6D1E9E70FF2E1028A6118690028EFD06D
:1025A00000F006F841F49071FFF74BFDF8D1DBE73E
:1025B000196851E8001F1A687047186800F108018F
:1025C00051E8001F00F10804704710B500F00EF844
:1025D000FCD100F015F8FCD1C16E00F025F82021E7
:1025E000C0F88C100022C266426710BD016851E835
:1025F000002F0B4622F4907243E800210029704717
:10260000016801F1080252E8002F01F10804DFF827
:1026100044140A4044E800210029704700000000EB
:102620000100001020010004012909D1026852E8CC
:10263000002F036822F0100243E800210029F5D1A1
:102640007047106800F1080454E8004F00F10806D4
:1026500070470000C06D0021A0F85E1000F00FBCB4
:10266000010002000400060008000A000C0010002F
:10267000200040008000000138B500F04DF81ED168
:102680004B6A9188846D0B402370816D4B1C00F068
:1026900049F818D100F04DF800F060F8FCD100F0D6
:1026A0006AF80BD10023136100F04EF8FCD10168E9
:1026B000CB69DC0644BF10230B6279E07DE08869BA
:1026C00040F00800886131BD38B500F025F81ED112
:1026D0004B6A9188846D0B402380816D8B1C00F0C8
:1026E00021F818D100F025F800F038F8FCD100F0FE
:1026F00042F80BD10023136100F026F8FCD10168E9
:10270000CB69DC0644BF10230B6251E055E08869B9
:1027100040F00800886131BD00F15C020168136B74
:10272000222B7047836551884B1E538051880029A6
:102730007047036853E8003F046823F4907344E84B
:1027400000310029F5D17047016851E8003F0C467F
:1027500023F0100344E8003100297047016801F1BB
:10276000080353E8003F01F108055B085B0045E8FA
:10277000003100297047202111630023936100215B
:1027800051610168374B99420CD049680B0209D559
:10279000016851E8003F0C4623F0806344E80031B3
:1027A0000029F5D11169012970470000F369FFCFB5
:1027B0001188BDE8344000F063BBBDE8324000F052
:1027C000B9BA00002DE9F84300F00CF946D1A08910
:1027D000002835D0B80633D500F0B0F80870A86DE1
:1027E000421C00F0D9F812D0F90748BF5FEAC8527E
:1027F00000F0AAF803D5F10701D500F0C5F800F004
:10280000ACF820B1284600F03AFB002060636088F5
:102810000028DFD100F035F8FCD100F0D3F8FCD16E
:1028200000F0FEF809D100F0EBF844BF102101627E
:102830002188284600F024FB02E0284600F07AFABE
:10284000608868B1A18988420ADA00F0AEF8FCD14C
:102850008148A06100F08EF8FCD101E000F00CF896
:10286000BDE8F18300240046FFF4FF110038014069
:102870000024F400E00C0246816941F00801816106
:102880007047296851E8001F2A6821F4807142E8E6
:1028900000100028704700002DE9F84300F0A2F86E
:1028A00046D1A089002835D0B80633D500F046F8C7
:1028B0000880A86D821C00F06FF812D0F90748BF9D
:1028C0005FEAC85200F040F803D5F10701D500F0E7
:1028D0005BF800F042F820B1284600F0D0FA002062
:1028E000606360880028DFD1FFF7CBFFFCD100F0E8
:1028F00069F8FCD100F094F809D100F081F844BFE8
:10290000102101622188284600F0BAFA02E0284628
:1029100000F010FA608868B1A18988420ADA00F0F4
:1029200044F8FCD14D48A06100F024F8FCD101E04E
:10293000FFF7A2FFBDE8F183004400402968486A20
:10294000A96D09EA0000704705D501210162606B9D
:1029500040F001006063B8077047780708D5F107B9
:1029600006D52A6804201062606B40F002006063A4
:10297000606B7047296851E8001F2A6841F0200108
:1029800042E80010002870472A6802201062606B3D
:1029900040F0040060637047AA656088411E618052
:1029A0002868C76917F0070F7047286800F1080208
:1029B00052E8001F00F1080921F0805149E8001099
:1029C00000287047286800F1080151E8001F00F155
:1029D00008032048014043E8001000287047000029
:1029E00000FD0F000546286805F15C04B4F804906A
:1029F000C7690146D1F800808668216B222970479B
:102A000000212161286850E8001F024621F01001D2
:102A100042E800100028F5D12868C169CA0670474D
:102A2000202020630021A1610020606128680C49FA
:102A300088420CD04068010209D5286850E8001F80
:102A4000024621F0806142E800100028F5D120699B
:102A500001287047FEFFFFEF79260008C92600080D
:102A60000024004610B5DFF82843DFF8280300F003
:102A70004BF822626262A26262662046FFF7AAF801
:102A800008B100F00DFE0021204600F031FE08B133
:102A900000F006FE0021204600F035FE08B100F0EF
:102AA000FFFD204600F006FE18B1BDE8104000F022
:102AB000F7BD10BD10B5DFF8E042DFF8E00200F02E
:102AC00023F8E26122626262A2622046FFF782F886
:102AD00008B100F0E5FD0021204600F009FE08B134
:102AE00000F0DEFD0021204600F00DFE08B100F0F0
:102AF000D7FD204600F0DEFD08B100F0D1FD00F06A
:102B0000E3F82046012225E120600C204FF4E1315A
:102B1000002260616160A260E2602261A261704790
:102B200070B596B004461421684600F03FFE40217F
:102B300006A800F03BFE20689649994C994D9A4EA4
:102B4000884223D14FF40072002106920F9106A80B
:102B500000F030FE08B100F0A3FDF06940F0400045
:102B6000F061F06900F0400000F05AF84FF40061A5
:102B700000F04DF8082100F043F800224FF4806087
:102B800000F033F8082200F036F82CE08349884240
:102B900029D1012200210692079106A800F00AFE21
:102BA00008B100F07DFDB06940F48040B061B069CB
:102BB00000F4804000F034F84FF4805100F027F822
:102BC000072100F01DF800224FF4807000F00DF88E
:102BD000072200F010F8002200212E2000F0FBFE5A
:102BE0002E2000F01FFF16B070BD0221029203924A
:102BF00000900191704704926946204600F072BF30
:102C00000222049101926946284600F06BBF02F04F
:102C100001020592059800910021029103917047ED
:102C200005900598316841F002013160326802F088
:102C3000020205920598316841F001013160326865
:102C4000704738B50168534B584A554C554899421E
:102C50000ED155684FF4006125F04005556000F035
:102C6000F8FF20464FF48061BDE8344000F0F1BF2A
:102C70004A4B994211D1116821F4804111604FF4FF
:102C8000805100F0E6FF4FF48071204600F0E1FF34
:102C90002E20BDE8324000F0D0BE31BD38B504462C
:102CA0003D4D2846FEF7DAFF6C602846FEF792FF9E
:102CB00010B14FF0FF3032BD00F006F80122284677
:102CC000FFF741F8002032BD394901F2DC50002203
:102CD0000260704710B5364C40F2DC51204600F0DF
:102CE00065FD04F2DC500022026010BD0A46014678
:102CF00080B54FF0FF332848FEF7D5FF08B14FF0FD
:102D0000FF3002BD2A4910B501F2DC525388148805
:102D1000A3420CD0C95C0170508840F2DC51401CC9
:102D200083B28B42A8BF00205080002010BD4FF01E
:102D3000FF3010BD10B51E49B1F8DC3540F2DC544F
:102D40005B1C9AB2A242A8BF0023A1F8DC359BB25B
:102D500001221944BDE81040FEF7F5BFF8B50C4656
:102D60001546012818BF022802D04FF0FF30F2BDEF
:102D70000026074F07E04FF0FF330122A119384624
:102D8000FEF791FF761CAE42F5D32846F2BD000057
:102D90002809002000240046BC090020003801401A
:102DA00000000242000402428C0C0246A40C0246BF
:102DB000D800002001484068704700BF0000002094
:102DC00070B50446FFF7F6FF06462CB304F14C0538
:102DD000287A022802D02021E9601BE0206841699E
:102DE00041F00401416105202872206801698A04CC
:102DF00014D4FFF7DFFF801B0628F6D3E868032111
:102E000040F01000E86029722879010602D5A96A0D
:102E10000120087300202870012070BD416941F035
:102E2000020141610420287222684FF4FE41012012
:102E3000D16000F018F80020287070BD30B100F1AA
:102E400054010A78022A03D02020486001207047EC
:102E500004220A700068416941F4005141F0040104
:102E600041610020704728722979080605D5A86AB3
:102E700001210173226800219164704700007047AE
:102E800070477047704770472DE9F84F040044D0F1
:102E9000DFF80477D7F81C90D7F828A0207809F03D
:102EA0000C090AF00305C1072AD5B9F1080F04D0AF
:102EB000B9F10C0F08BF032D62D1606800282CD037
:102EC000B9F1080F1CD13968A068012221F48811DA
:102ED000014341F4803139603868DFF8DC16DFF8EF
:102EE000D436000D00F001008240B1FBF2F1DFF8B2
:102EF000C0261160186800F027FF002840F0E98123
:102F00002078810712D5B9F1000F04D0B9F10C0F68
:102F100008BF022D57D12069002800F0DA813869F6
:102F2000616920F4F81040EA014038612078DFF848
:102F30008C86DFF88C56010740F1C08028684FF07E
:102F4000000A41070AD428684FF0010A40F0040043
:102F50002860296801F0040100910098D8F8001059
:102F6000C80751D400F0DDF90646D8F80000C107C3
:102F70004AD4FFF71FFF801B0328F6D303207FE10D
:102F8000606888B13A68A16822F488121043084347
:102F900000F0C4F9064638688103B1D4FFF70AFF90
:102FA000801B6528F7D3E9E7386820F4881000F023
:102FB000B5F9064638688103A2D5FFF7FBFE801BF2
:102FC0006528F7D3DAE7206978B1396841F4807170
:102FD0003960FFF7EFFE0546386841059FD4FFF7DB
:102FE000E9FE401B0328F7D3C8E7386820F4807057
:102FF00000F094F905463868410597D5FFF7DAFEE9
:10300000401B0328F7D3B9E7EE6DA069002843D031
:1030100040011AD5E16906F08050814211D031019A
:103020000FD526F08066EE65FFF7C4FE8346E86D97
:10303000010106D5FFF7BEFEA0EB0B001528F6D365
:103040009CE726F08050E6690643A0690643EE65DA
:10305000FFF7B0FE0090B346A669E86D10EA460F90
:1030600006D1FFF7A7FE0099401A1528F4D385E78B
:1030700086F010562BEA060BC5F85CB0FFF79AFEF7
:103080008346E86D10EA460F16D0FFF793FEA0EBDB
:103090000B001528F5D371E726F01056EE65FFF703
:1030A00089FE0646E86D10F0904F05D0FFF782FECE
:1030B000801B1528F6D361E700F028F9217848072E
:1030C0006CD529684FF0000A48070AD429684FF0E8
:1030D000010A41F004012960286800F00400009012
:1030E0000098D8F80010C8070CD400F01AF906466A
:1030F000D8F80000C10705D4FFF75CFE801B032849
:10310000F6D33BE7E06841F2893828B3E96D21F056
:1031100080010843E865FFF74DFE0646E86D81072C
:1031200005D4FFF747FE801B4045F7D326E7207BF9
:10313000010608D5E86D01052ED4FFF73BFE801B84
:103140004045F7D31AE7E86D010525D5FFF732FEB4
:10315000801B4045F7D311E7E86D20F08100E8655A
:10316000E86D20F00400E865FFF724FE0646E86DF0
:10317000810705D5FFF71EFE801B4045F7D3FDE60E
:10318000E86D010608D5E86D010505D5FFF712FECB
:10319000801B4045F7D3F1E600F0B8F8206A00281C
:1031A0006DD0B9F10C0F6DD00228386820F0807016
:1031B000386053D1FFF7FEFD0546D7F800A0FFF7B2
:1031C000F9FD401B0328E6D25FEA8A10F5D4626A53
:1031D000032A07D14FEA1A51DFF8DC0301F001019D
:1031E000C84001E0DFF8C403A36ADFF8D813B0FBDE
:1031F000F3F088422CBF0C210021D7F82890DFF88B
:10320000C8035B1E00EA09000243114341EA03219F
:1032100041F48021B962E06A216B401E491E40EAF8
:103220004120616B491E40EA0140A16B491E40EA02
:1032300001607863E06B10B100F062F8B862386842
:1032400040F0807000F06AF804463868810116D4B6
:10325000FFF7B0FD001B0328F7D38FE6FFF7AAFDA9
:1032600004463868810105D5FFF7A4FD001B03283B
:10327000F7D383E6B86ADFF854130840B862002039
:10328000BDE8F28F012824D0B86A796B636A00F038
:1032900003029A4201BFC0F30220401CA26A90427E
:1032A00017D1E26AC1F30800401C904201BFC1F38C
:1032B0004620401C226B90420BD1626BC1F306404A
:1032C000401C904201BFC1F30660401CA16B8842C4
:1032D00001D00120D4E7B86BE16BC0F3CC00814290
:1032E000CDD0B86A20F01000B862FFF763FD054644
:1032F000FFF760FD401BFBD0E06B00F001F8BDE77D
:10330000C000B863B86A40F010007047BAF1000F0F
:1033100003D0286820F00400286070473860FFF769
:1033200049BDD8F8001041F00101C8F80010FFF7BE
:1033300041BD2DE9F0410400884637D0DFF89052B6
:10334000286800F00F00404509D22968090948EAB9
:1033500001112960286800F00F00404526D121782E
:10336000880609D5DFF840221368A169E06923F0D7
:1033700017030B43034313602178DFF81C72C8075F
:1033800042D53868616803290CD180016BD5F96991
:1033900001F00C010C290CD0B96A012060F3155121
:1033A000B96206E0022902D1800302D45BE0410544
:1033B00059D5FA696068920840EA8202FA61FFF71B
:1033C000F9FC06466068F96901F00C01B1EB800F69
:1033D00008D0FFF7EFFC801B41F289318842F1D31E
:1033E000032052E003280FD1B86A20F48010B8629D
:1033F000FFF7E0FC0646B86A410205D4FFF7DAFCA5
:10340000801B0B28F7D3EBE7396A2268002093076B
:1034100004D5C908C800A16801430120530704D599
:1034200021F07000E16801430120120705D52069F1
:1034300021F4E06141EA001100E000B13962207836
:10344000C10644BF60697862296801F00F018845B0
:103450000BD22868000948EA00102860296801F0AA
:103460000F01414501D001200FE000F010F83A6A49
:1034700058494F4B02F00702895CC84018604D481C
:103480000068BDE8F04100F05FBCBDE8F081424952
:10349000C86910F00C0001D144487047082818BFD3
:1034A00000F036B809684448090D01F00101C84030
:1034B000704780B5FFF7EBFF47490968454A3C4B29
:1034C00001F00701515CC840186002BD80B5FFF7EC
:1034D000F0FF414A0CE080B5FFF7EBFF3E4A13686E
:1034E0003E49C3F3022207E080B5FFF7E2FF3C4A02
:1034F00013683A49C3F30212895CC84002BD10EE5A
:10350000100A491CB0FBF1F010BD3648046807E012
:1035100010B5FFF7FAFFBCEEC00AC4F30661EEE790
:103520001D48416BC1F30801491C00EE101A816A65
:10353000B8EE400AC1F30222521C00EE902AF8EEC7
:10354000600ACA0643BF826BC2F3CC0201EE102AA6
:103550009FED121A01F00301B8EE411A022902D0C0
:10356000032903D00DE0DFED0E1A0CE000681249CC
:10357000000D00F00100C14001EE901AF8EE611A52
:1035800001E0DFED061AC1EEA00ADFED061A01EE3A
:10359000210A20EE800A7047000C0246000000005D
:1035A0000024744B00000039000E02460024F40091
:1035B0000C000020080000200048E801280802460E
:1035C000940C024601127A00E0F8FFFFFCFFF8FFBE
:1035D00000200240A0450008200C0246705F000851
:1035E000240C0246340C024680B500F0F7FB00F0D4
:1035F00013F800F00DFCFFF735FAFFF75BFA00F067
:10360000A9FC00F005FD00F013FD00F076FC00BF02
:1036100024A000F0EBFEFEE780B598B0402108A89A
:1036200000F0C4F82021684600F0C0F84FF4803064
:1036300000F0F0FE08B100F033F800220A920F9279
:103640004FF480310322099111924FF080610822DA
:1036500009200E91139208900221002210911291DC
:10366000149115911691179208A8FFF70DFC08B157
:1036700000F016F83F2100910021032202910491ED
:1036800001920421002206910392059207920121E2
:103690006846FFF74EFE08B100F002F819B000BD11
:1036A00072B6FEE74C5445205445535420444F4EC7
:1036B000450D0A0010B500F184010A78012A01D1F4
:1036C000022010BD01220A7024234B600268136897
:1036D000146864086400146000224266006823F0E5
:1036E0000053202203604A6000230B70002010BDAD
:1036F00070B500F01FF801D1022070BD00F020F875
:1037000022F0604209E070B500F014F801D1022007
:1037100070BD00F015F822F0606211438160204610
:1037200000F01CF8206820210022066069602A70E1
:10373000002070BD044604F18405287801287047F4
:103740000120287024226A602068066802685208F6
:1037500052000260206882687047000030B5416EF8
:1037600011B90121012214E0016800BF0FF22C04FD
:103770000CA38A688968520E02F00702490F655C43
:10378000A45C595C9A5CED00E40095FBF1F194FBBC
:10379000F2F268304180028030BD00000101010377
:1037A000070100000804020408010101002200F0E2
:1037B0005FBE00002DE9FC4706463078DFF8EC716B
:1037C000C10705D53A687068920840EA82023A60FB
:1037D0003178880705D53968B06821F00C010143BC
:1037E00039603178480705D53968F06821F44061BF
:1037F000014339603178080705D53968306921F40B
:103800004021014339603178C80605D539687069AF
:1038100021F44011014339603178880605D53968B3
:10382000B06921F44001014339603178480605D57B
:103830003968F06921F00041014339603168DFF8EF
:103840007041C8050DD57968306A21F440510143B3
:103850007960316AB1F5405F03D1206840F40030EF
:1038600020603168880505D5B968706A890840EA22
:103870008101B9603168480505D5B968B06A21F0A1
:1038800018010143B9603168080505D5B968F06AC7
:1038900021F0C0010143B9603168C80405D5B96899
:1038A000306B21F440610143B960316888040DD563
:1038B000B968706B21F4E0410143B960716BB1F5F7
:1038C000005F03D1206840F48030206031684804F4
:1038D00058D5D7F81090B06B4FF0000809F4407934
:1038E00081454FD0E16E48070AD4E16E4FF00108E0
:1038F00041F00401E166E06E00F0040000900098E1
:10390000DFF8B050286840F001002860FFF752FA55
:1039100082462868C10707D4FFF74CFAA0EB0A00DB
:103920000228F6D903203FE03869B9F1000F20F4EE
:10393000407009D0B9693A6942F480323A613A6913
:1039400022F480323A61B961B16B01433961DFF829
:10395000681011EA00090ED0FFF72CFA0546386905
:1039600010EA490F07D1FFF725FA401B41F28931D0
:103970008842F4D3D6E7B8F1000F03D0E06E20F010
:103980000400E066306801040DD53A69F06B22F45A
:10399000402202433A613969F06B01F440218142CF
:1039A00018BF012000D10020BDE8F687E00C0246D8
:1039B000280C02462808024601000024414B1968E1
:1039C0004FF6FF020002114000F4E06008433E4958
:1039D00008431860704770B53A4B1C68C4F3022363
:1039E0000124C3F10705052D2EBF0F2504FA05F5A7
:1039F0006D1E1E1D072E34BF0023DB1E294099407B
:103A000004FA03F35B1E1A4011430901020002D4B9
:103A10002E48815470BD2E4B02F00F021A4402F85A
:103A2000041C70BD010007D4012200F01F018A4070
:103A3000284B400943F82020704701000BD4012295
:103A400000F01F018A40244B400943F82020BFF3B7
:103A50004F8FBFF36F8F7047401EB0F1807F07D24A
:103A60001E49486000228A600B6843F003030B6024
:103A7000B0F1807F8041C043C00F70471849174A9A
:103A800004281ED8DFE800F00811141D0300106898
:103A900040F0040010607047136823F004031360C3
:103AA000086820F44000086070471368012001E0B6
:103AB0001368022023F0040313600A6860F397522E
:103AC0000A6070470CED00E00000FA0500E400E039
:103AD00018ED00E000E100E080E100E010E000E02F
:103AE000E00C02462DE9F04F4FF0000C924A934B48
:103AF000DFF84C824FF00F0906460F46A2E0012482
:103B000004FA0CF414EA010058D04FEA4C010325E2
:103B10008D406FEA050E7D6805F0030ABAF1010FCA
:103B20001CBF05F00305022D13D1B568D7F80CA012
:103B30000EEA05050AFA01FA4AEA0505B560756854
:103B400025EA04047D68C5F3001505FA0CF52C433D
:103B500074603D79BC6805F00305032D08BF012C96
:103B600005D0F5688C400EEA05052C43F4603C79DD
:103B700004F00304022C14D14FEADC0406EB8404A5
:103B8000D4F820A04FEA8C0505F01C0509FA05FBC6
:103B90002AEA0B0AD7F810B00BFA05F545EA0A0530
:103BA000256234680EEA04053C7904F0030404FA43
:103BB00001F129433160796811F4403F40D04FEA68
:103BC0009C01DFF880A158F821E04FEACC040AEA12
:103BD000962A04F0180409FA04F52EEA05050AFAF3
:103BE00004F444EA050E48F821E0D3F800E07C68CC
:103BF000C14301EA0E0EE50248BF40EA0E0EC3F8CB
:103C000000E0D3F804E07C6801EA0E0EA50248BF8C
:103C100040EA0E0EC3F804E0D2F804E07C6801EA42
:103C20000E0EA50348BF40EA0E0EC2F804E0D2F81B
:103C300000E07C6801EA0E01E40348BF0143116023
:103C40000CF1010C396831FA0CF07FF458AFBDE883
:103C5000F08F2DE9F04F02460027384BDFF8D8806F
:103C60004FF00F09DFF8D8A053E0012000FA07FC5D
:103C70001CEA01004CD04FEA970EDFF8C8B05AF8A2
:103C80002E60FD000BEA922B05F0180509FA05F4E9
:103C900026400BFA05F5AE4216D1D8F80050C043C5
:103CA0000540C8F80050D8F804600640C8F8046021
:103CB0005D6805405D601E68304018605AF82E004F
:103CC00020EA04044AF82E4003207C00A040146837
:103CD000FD0802EB850E04431460DEF82040BD00B1
:103CE00005F01C0509FA05F5AC43CEF82040D2F8E2
:103CF00008E0C04300EA0E0EC2F808E0546824EA67
:103D00000C0CC2F804C0D2F80CC000EA0C00D06061
:103D10007F1C31FA07F0A8D1BDE8F08F0AB18161AC
:103D2000704781627047426901EA0203914341EAA8
:103D30000341816170470000802002460020024656
:103D4000602002467F7F2F00F8B504461F4D28787B
:103D5000002100282ED01E4A12681E4B1E687707CD
:103D600002D54FF47A710DE01B4B1B6813F440032E
:103D700006D0B3F5800F08D0B3F5000F0ED015E0D4
:103D80004FF4FA51B1FBF0F00EE04FF47A72B2FB4F
:103D9000F0F24FF4FA43B3FBF2F107E04FF47A711B
:103DA000B1FBF0F04FF40042B2FBF0F10846FFF730
:103DB00053FE08B10120F2BD002221464FF0FF3032
:103DC000FFF709FEAC600020F2BD00BF000000203C
:103DD0000C00002010E000E0E00C024680B50B482B
:103DE000016841F4807101600320FFF7E7FD00F0F6
:103DF00063FB0420FFF742FE0F20FFF7A5FF08B189
:103E0000012002BD00F0D0FB002002BD00200240D6
:103E100038B586B0142101A8FFF7C8FC46480168F0
:103E200048F29105454C41F002010160026802F040
:103E3000020200920099026842F0010202600368E7
:103E400003F00103009300990268294642F004023E
:103E500002600068002200F004000090009800F06A
:103E600049F801210291002201950392049201A9CF
:103E70002046FFF737FE07B030BD012200E00022E8
:103E800080212E48FFF74ABF10B52C4C012210218B
:103E900000F030F82A4800F0A9FA00F055F800F0D8
:103EA00027F8642000F0A0FB012200F022F8012294
:103EB00000F04BF8C82000F097FB00F019F84FF421
:103EC000AF7000F091FB00F03FF8642000F08CFB35
:103ED0000C24FFF7D2FF4FF4FA7000F085FBFFF7D8
:103EE000CEFF4FF4FA7000F07FFB641EF1D110BDDD
:103EF000002201212046FFF711BF10B5114800F044
:103F000075FA0E4C00F020F8642000F06DFB0122E1
:103F100000F01BF84FF42F7000F066FB00F014F86F
:103F2000FFF7ABFF1E244FF47A7000F05DFB641EB8
:103F3000F9D1BDE81040A2E78C0C02460004024211
:103F40006C5E0008905E000800224FF4004120469D
:103F5000FFF7E4BE18B587B01C220021684600F0C8
:103F600057FB284C28482060FF20E0604FF080403D
:103F700000217F22E0616160A26021616161A16135
:103F800021626162204600F04DFB08B1FFF788FB1B
:103F9000002100910391049105916946204600F0AB
:103FA00042FC08B1FFF77CFB00220021204600F014
:103FB000F7FB08B1FFF774FB08B010BD10B590B067
:103FC000044640220021684600F022FB21680E4A88
:103FD000914215D14FF480434FF4007100930E913C
:103FE0006846FFF7E7FB08B1FFF75AFB074801688F
:103FF00041F400110160006800F400100090009886
:1040000010B010BDA00A002000780046A80C02469F
:1040100080B5002000F026FC08B1FFF741FB00F05E
:104020002DFC18B1BDE80140FFF73ABB01BD00000F
:104030002DE9F04F9BB0002000900027DFF8C4521C
:104040000FF234360FF21C3B0FF204380FF2EC295A
:10405000DFF8B4A2322000F0C7FAFFF715FF78208E
:1040600000F094F804460A22514601A800F016FC1C
:104070000146484600F0BAF900F084F801A800F0C3
:1040800031F901A9404600F0B1F900F07BF801A830
:1040900000F024F901A9584600F0A8F900F072F8E0
:1040A00001A800F02AF901A9304600F09FF900F0BC
:1040B00069F801A800F01DF901A90FF2C82000F06D
:1040C00095F9652101A87F1CFFF770FBFF2C4FD0ED
:1040D0000A2C54D0002C1DD1284600F087F900F09E
:1040E00051F8684600F0E6F80098632808D04100CF
:1040F0000246713949B205F12C0000F077F903E06E
:1041000005F15C0000F072F970A000F06FF905F5A0
:10411000807015E0FBD0012C17D0022C1FD0032C8F
:1041200023D0042C18BF052C0FD00A2C27D0FF2C2D
:104130001ED021460FF2782000F058F905F5CE7018
:1041400000F054F9032F85DB0CE000F0AFF805F127
:10415000840000F04BF900201BB0BDE8F08F05F1A2
:10416000B000EDE74FF0FF30F6E705F1D800E7E7E4
:1041700005F5947000F03AF905F5B070E0E70FF23C
:104180001020DDE7652101A8FFF710BB2DE9F04FF6
:1041900085B0002603968DF81060DFF86CB182467A
:1041A000FEF708FE0546DFF86411584600F085FE6C
:1041B000DFF85C01DFF85C11DFF85C21029001910F
:1041C0000092DFF85831DFF85821DFF858115846CF
:1041D000FF274FF47A7400F047FC04FB0AF402282E
:1041E00060D1584600F064FC022855D1FEF7E2FD8C
:1041F000401B39A7DFF830814FF6FF790EE03846D3
:1042000000F0F4F805E0002EF9D1404600F0EEF899
:10421000012600F04BF8FEF7CDFD401BA04201D374
:10422000CA4511D103A9584600F078FD0228F2D101
:1042300003986328E7D04100713949B20FF290101A
:1042400000F0D4F800F032F8FEF7B4FD401B9DF901
:10425000107004E000F02AF8FEF7ACFD401BA0420D
:1042600001D3CA450DD1584600F06FFD022808D091
:104270007F1C78B20128EDD1584600F084FD022859
:10428000E8D0584600F09EFD0746012818BF0528D3
:1042900008D1FEF78FFD05E0082802BF9BF8D27019
:1042A000032F1327384605B0BDE8F08F4FF47A701E
:1042B00000F09AB9014610B500F00BF800F02EFDA1
:1042C000022808BF0024204610BD00000D0A00008F
:1042D00001210D48022470472E00000080B56422A1
:1042E000124902E080B51022114900F0D7FA0020EF
:1042F00002BD80B514220F49F7E780B510220E49A0
:10430000F3E70000D05A0008B8060020B52D0008D9
:10431000D52C0008052D0008ED2C00089D2C000868
:104320005D1C0008B52A0008E85D0008F4060020BE
:10433000C2060020C0070020580700204D6F64759A
:104340006C65204E616D653A2025730D0A000000F2
:1043500050726F647563742049443A2025730D0AC6
:104360000000000046572056657273696F6E3A2050
:1043700025730D0A00000000494D45493A20257378
:104380000D0A000049434349443A2025730D0A00B1
:104390000D0A203E3E3E2053494D206973206E6F2A
:1043A0007420494E5345525445440D0A0D0A0000ED
:1043B0000D0A203E3E3E204D6F64756C65205349CA
:1043C0004D204572726F723A2025640D0A0000007C
:1043D0000D0A5369676E616C204C6576656C3A20F6
:1043E00025642064426D0D0A000000000EB4C0B5C3
:1043F000024603A800210190009101AB012104486D
:1044000078440C30FBF7ADFE06BC5DF810FB00BF36
:10441000391B000010B5134A116B01F48031814241
:104420001BD01168104B21F48031084310601C68C8
:1044300032200E494443B4FBF1F1491C084601E027
:1044400068B1401E13681C04FAD540B101E031B1D7
:10445000491E106B0304FAD509B1002010BD0320DA
:1044600010BD00000C0802460C00002040420F0066
:1044700000B500BF130096469446103928BFA0E847
:104480000C50FAD85FEA417C28BF0CC048BF40F806
:10449000042BC90728BF20F8022B48BF00F8012BC6
:1044A00000BD000037480168374A41F470010160DF
:1044B000364810607047000030B53549CB69354843
:1044C000354A03F00C03082B02D00C2B07D04BE02D
:1044D00010460A68120D02F00102D04044E08B6AD7
:1044E0004C6BC3F302256D1C00EE105AC4F3080593
:1044F000C4F30664641C6D1C01EE104A00EE905A71
:10450000DC0607D58C6BC4F3CC0401EE904AFBEEBD
:10451000E91A01E0DFED1A1A03F00303022B02D0BF
:10452000032B03D00AE002EE100A09E00868000D30
:1045300000F00100C24002EE102A01E09FED102AB7
:10454000B8EE422AB8EE400AF8EE600A82EE000A9F
:1045500070EEA10A20EE200AF8EE410A80EE200A51
:10456000BCEEC00A10EE100A0C4A1060096A00BFC7
:104570000BA301F00701595CC840106030BD00007A
:104580000000000088ED00E008ED00E000000008F9
:10459000000C02460024F4000048E8010C00002052
:1045A000000000000102030480B50E48816841F05C
:1045B00004018160816801F00401009100990268A2
:1045C000002142F4801202600068002200F4801092
:1045D000009000984420FFF7FEF94420BDE8024017
:1045E000FFF720BA8C0C024638B50446FEF7E2FB12
:1045F000054614F1010F02D0044908780419FEF7AA
:10460000D9FB401BA042FAD331BD00BF00000020FF
:1046100010B5044610460A460146204600F0EEFC5E
:10462000204610BD70B504460120002C49D004F18D
:104630002C05697821B9002028702046FFF7BEFCC0
:1046400002216970DFF850613068C10636D4CA2093
:10465000B0615321B161204600F052F8010028D129
:10466000F168DFF838010140F160F26860682169A3
:104670000243A0690A430243F260E168A06841EA8C
:10468000004171603268616AA06A22F4F8520A43FC
:1046900002433260204600F057F8010009D1F36868
:1046A000226AE16923F06043134362690B431343B9
:1046B000F360FF21B161020003D100E0002001217D
:1046C000697070BD84F82D0070BD70B50446324D20
:1046D000286820F020002860FEF76CFB064628685A
:1046E00081060BD4FEF766FB801B40F2E93188425D
:1046F000F5D32868810601D40320E3E7002070BDCC
:10470000F8B50546244C2068002641061AD42068D6
:1047100040F080002060FEF74DFB074603E00320D9
:10472000032685F82D00216848060BD4032E09D0F6
:10473000FEF740FBC01B40F2E9318842F3D320680A
:104740004106ECD53046F2BD70B50446124D2868DE
:10475000002620F080002860E968880608D42046FA
:10476000FFF7B3FFA0B1032084F82D0003260FE06C
:10477000E86820F02000E8602046FFF7A6FF18B1A7
:10478000032084F82D000326E86840F02000E8604C
:10479000304670BD000000000C780046BFFF8FFB64
:1047A0002DE9F04100F12C0630780C461546012821
:1047B00008BF02202FD00120307002217170DFF875
:1047C0009870F86820F48060F8603968480614D45E
:1047D000FEF7F0FA8046386841070ED4FEF7EAFA91
:1047E000A0EB080000F01BF8F5D33868410704D4AB
:1047F00003207070002131700DE0F8680121C008BD
:1048000045EAC005FD60BC60F86840F48060F8606F
:10481000717000203070BDE8F081A0EB090040F21B
:10482000E9318842704710B50A6848680C4B02436A
:104830001A608C68CA688869084B144304435C603A
:104840001A680869496922F0FF12024342EA0142EC
:1048500000201A6010BD00000C780046207C004645
:104860001C78004610B500F010F801D5012010BDED
:10487000136823F004031943116010BD0648016852
:1048800041F00101016000207047034A13680146AE
:104890000020DC07704700000004034001B55AB156
:1048A00011F8013B521E00F8013B03B1F8D1110091
:1048B0001CBF002200F0A2FB01BD000070B5024643
:1048C00015780023002400202D2D0AD10123521C2D
:1048D000012406E012F8016B0A25641C05FB006048
:1048E00030381578303D0A2DF4D301B10C7003B186
:1048F000404270BD002381423CBF4FF0FF331B1A82
:10490000591A4018101870472DE9F24F82460AF5DF
:10491000B2709AB0416893461C46249F8847019024
:104920000BF10F024FF47A5042434FF4E13100266D
:1049300092FBF1F0B84238BF384624900025DFF8EA
:10494000A4750DF138090DF1080868206843391D78
:1049500029F815600844FCF7D1FB28F815006D1CF8
:10496000172DF2DB5FEA0B0008BF002C51D04FF48B
:1049700080710AF5B670FEF719FF0AF5B27A02E007
:10498000521C172A1ADBDAF8040080470146249AE1
:104990000198FFF7AFFF002836DDDAF8001068460F
:1049A00088470028EFD19DF800001A998855761C99
:1049B00036B25FEA0B0224D10022682101FB02F02B
:1049C00039F812E09DF800C03B189E449EF8045050
:1049D000AC451CBF002529F8125039F812509DF83B
:1049E00000E02B441B799E45CAD16D1C29F812505A
:1049F00038F81230ADB29D42C2D338580442BFD00D
:104A00000BE05E45BFDB04E0BBF1000F03D0002EDE
:104A100001DD304601E04FF0FF301BB0BDE8F08F04
:104A20002DE9FC4105460C0016461F466FF00108B3
:104A300008BF4FF4AF743046FCF760FBD5F8602137
:104A400081B23046904700280BD4C820FFF7CCFD38
:104A500000943B46002205F5B6712846FFF754FF47
:104A600080464046BDE8F681F0B570B10C000CD030
:104A700014000AD01C0008D0059C250005D0069D16
:104A80002E0002D0079E370001D14020F0BD00F576
:104A9000A87001604260836004614561C6600220C5
:104AA000F0BD002204F5B67120462DE7000000009D
:104AB0002DE9FC4780460020202788F83B0100258F
:104AC000002200230A214143414401F59F71401C0B
:104AD0000A704B704D808A80CB800028F2DD08F58B
:104AE000A874E068804721688847002840F0068164
:104AF000A06940254FF0000A8047814681A6A06941
:104B0000804701464FF4FA724846FFF7F3FE00284B
:104B10000AD542233246642100F0FAF80546A0691E
:104B20000AF1010A804781464FFA8AF00A286ADAB8
:104B3000022DE4D1404600F073F9064608F5A47151
:104B4000404600F073F9054642230FF2A83200F008
:104B5000DDF8814642230FF2A4324FF47A714046C9
:104B60002E43FFF75DFF49EA0606064342230FF294
:104B700094324FF4AF7100F0CBF8064308F5B675E8
:104B80000FF29829022E46D142230FF2843200F010
:104B9000BDF8022806D100F0BDF801460A224046C1
:104BA000FFF77CFE42230FF2743200F0AFF80228C8
:104BB00007D100F0AFF80146322208F10A00FFF7F2
:104BC0006DFE42230FF2603200F0A0F8022807D1F8
:104BD00000F0A0F80146642208F13C00FFF75EFEF9
:104BE00042230FF250324FF4AF7100F091F80646B5
:104BF000022E10D100F08EF80146322208F1A000FA
:104C0000FFF74CFE09E0022D94D0DFF8DC02FFF73D
:104C1000EDFB04275EE0022E5CD1A06980470646CA
:104C2000A1698847801BB0F5FA6FF9D348F24204B6
:104C300023460FF20C3241F27C5100F069F8022851
:104C400035D10FF20831284600F0E1F9002841D0B3
:104C5000FF2088F8D20023460FF200324FF4AF71E4
:104C600000F056F8022807D100F054F8014632222D
:104C700008F1D600FFF712FE42230FF2EC224FF4A8
:104C8000AF7100F045F802280FD100F043F83A2147
:104C9000FCF708FA18B110F8011F2029FBD00146D3
:104CA000322208F58470FFF7F9FD022712E0B0F513
:104CB000004F0FD100F063F801230022294640463F
:104CC000FFF722FE01A908F26D10FFF7F7FD88F843
:104CD000D200082748F242030FF2982244F27401EE
:104CE00000F016F8022818BF20274FF01E081E20DB
:104CF000FFF77AFCB8F10108F9D100E01027384637
:104D0000BDE8F68741540D0A000000004FF47A71A7
:104D1000404685E64946284600F090B97CB500F04B
:104D20004CF80FF25C224FF4AF71FFF779FE0646A4
:104D3000022E08D10FF2542100F0BBF86946801D05
:104D4000FFF7BCFD2860304676BD38B5044694F8C0
:104D5000D2004025FF2810D148F242030FF234223E
:104D6000DFF8881100F0BAF8022805D000F007F843
:104D70000123FFF796FE00E00225284632BD4FF4DE
:104D80007A70009070471CB500F018F80FF21422EA
:104D9000DFF85C1101E044F27401FFF741FE0228E4
:104DA0000AD04FF47A7000900123002204F5B67106
:104DB0002046FFF7A9FD402016BD0D46044648F2E7
:104DC0004203704738B500F022F818D148F2420388
:104DD0000FF2DC1200F080F8022810D10FF2DC1183
:104DE00000F067F858B100F1090101226846FFF7A9
:104DF00055FD00F006F8684600F0E8F90546E8B20F
:104E000032BD022205A10DF10100FFF747BD0446A6
:104E100094F8D200FF25FF28704700000D0A00001B
:104E200042230FF2A8124FF4AF71F9E5F8B50C4622
:104E300042230FF2A0124FF4AF710546FFF7F0FDC9
:104E400005F5B67602280AD10FF29411304600F02B
:104E5000DEF80021801DFFF731FDC5F8480142232F
:104E60000FF284124FF4AF7100F033F80546022DB3
:104E70001BD10FF28011304600F0C9F8861D0021C9
:104E80003046FFF71BFD07460021B01CFFF716FD5B
:104E9000FFB2C0B2022F04D1022814BF01200320A8
:104EA00002E0022818BF002060602846F2BD0FF221
:104EB000141104F5B67000F0AAB808B10A0001D1C7
:104EC00040207047C0F868110220704760233A46BE
:104ED00041462846FFF7A4BD4FF4AF712046FFF7C7
:104EE0009FBD000048520008185E0008B030010065
:104EF00090D60200415456310D0A0000415445300D
:104F00000D0A000041542B434D45453D310D0A002B
:104F100041542B43474D490D0A00000041542B4397
:104F2000474D4D0D0A00000041542B43474D520D93
:104F30000A00000041542B4347534E0D0A00000065
:104F400041542B4350494E3F0D0A00002B4350491A
:104F50004E3A2052454144590000000041542B4331
:104F6000494D490D0A00000041542B49434349442F
:104F70000D0A000041542B4346554E3D310D0A00A9
:104F800041542B4353510D0A000000002B43535151
:104F90003A00000041542B43474154543D310D0A1F
:104FA0000000000041542B434F50533D300D0A0088
:104FB00041542B435245473F0D0A00002B435245B5
:104FC000473A00002B434F50533A000041542646C5
:104FD0000D0A000041542B4950523F0D0A000000B9
:104FE0002B4950523A00000041542B4946433F0D93
:104FF0000A0000002B4946433A0000004018491CB3
:105000001CBFB1F1010100F8012DF9D1704770B555
:105010000D462C7834B970BD11F8013F1678B342B3
:1050200006D0401C2146FCF73DF828B101462A462F
:1050300012F8013F002BEFD170BD000038B504001D
:105040000D460BD02946204600F0C7F804442078CE
:1050500048B90C4800210160002032BD09490C68A4
:10506000002CEFD132BD2946204600F0C7F82118A8
:10507000087810B1002201F8012B02480160204697
:1050800032BD00BFD00A00202DE9F84F84B00E4693
:1050900017460BB100221A600446A04601E008F151
:1050A000010898F8000000F0BAF80028F7D198F845
:1050B00000002D2816BF2B2818F8015B2B25002F88
:1050C000019603D4012F01D0252F03DB002E56D0EB
:1050D000346054E0002F0CDD102F04BF98F800005E
:1050E000302802BF98F8010040F02000782811D144
:1050F0000CE098F80000302818BF0A270AD198F869
:10510000010040F02000782803D1102708F10208A0
:1051100000E00827CDF80C8001E008F1010898F8BC
:1051200000003028F9D0064E7E4414364FF00009B6
:1051300006F12800CDF80880CA468DF800000CE082
:10514000800B000001469DF80000081ACA465FFA6D
:1051500080FB07FB09B908F1010898F8000000F08E
:1051600068F801463A4606F12800FBF7D1FF00280F
:10517000E8D10399414504D1019800B104600020B1
:1051800020E00299F05DA8EB0101091A002910D472
:1051900006DCB9EB0B0103D3B1FBF7F0504508D0A7
:1051A000AFF30080049808B1012101604FF0FF398E
:1051B00003E02D2D08BFC9F10009019808B1C0F81E
:1051C0000080484605B0BDE8F08F04E000E0000034
:1051D0000A220021F9E7002356E770B4044600E0F4
:1051E000641C23783BB10D462A7822B115F8016B77
:1051F000B342F9D1F4E7201A70BC704770B404468A
:1052000000E0641C23783BB10D462A78002AF8D0D0
:1052100015F8016BB342F8D1201A70BC704710B575
:105220000446FCF73DFC01462046096ABDE81040F3
:10523000084710B50446FCF733FC01462046896A4E
:10524000BDE8104008470000100000004F4B0D0A59
:10525000000000000000000000000000000000004E
:10526000000000000000000000000000000000003E
:10527000000000000000000000000000000000002E
:10528000000000000000000000000000000000001E
:10529000000000000000000000000000000000000E
:1052A00000000000000000000000000000000000FE
:1052B000080000003E0000000000000000000000A8
:1052C00000000000000000000000000000000000DE
:1052D00000000000000000000000000000000000CE
:1052E00000000000000000000000000000000000BE
:1052F00000000000000000000000000000000000AE
:10530000000000000000000000000000000000009D
:10531000000000000000000000400000434950521F
:105320005847455400000000000000000000000045
:10533000000000000000000000000000000000006D
:10534000000000000000000000000000000000005D
:10535000000000000000000000000000000000004D
:10536000000000000000000000000000000000003D
:10537000000000000000000000000000000000002D
:105380000000040043495053454E44000000000013
:10539000000000000000000000000000000000000D
:1053A00000000000000000000000000000000000FD
:1053B00000000000000000000000000000000000ED
:1053C00000000000000000000000000000000000DD
:1053D00000000000000000000000000000000000CD
:1053E000000000000000000000000200504F574580
:1053F00052454420444F574E0D0A00000000000063
:10540000000000000000000000000000000000009C
:10541000000000000000000000000000000000008C
:10542000000000000000000000000000000000007C
:10543000000000000000000000000000000000006C
:10544000000000000000000000000000000000005C
:10545000000009005244590D0A000000000000003D
:10546000000000000000000000000000000000003C
:10547000000000000000000000000000000000002C
:10548000000000000000000000000000000000001C
:10549000000000000000000000000000000000000C
:1054A00000000000000000000000000000000000FC
:1054B000000000000000000080000000636C6F73BB
:1054C00065642200000000000000000000000000F1
:1054D00000000000000000000000000000000000CC
:1054E00000000000000000000000000000000000BC
:1054F00000000000000000000000000000000000AC
:10550000000000000000000000000000000000009B
:10551000000000000000000000000000000000008B
:105520000001000043495052584745543A535543EF
:10553000434553530000000000000000000000003D
:10554000000000000000000000000000000000005B
:10555000000000000000000000000000000000004B
:10556000000000000000000000000000000000003B
:10557000000000000000000000000000000000002B
:10558000000000000000000000020000696E636F70
:105590006D696E672066756C6C220000000000006B
:1055A00000000000000000000000000000000000FB
:1055B00000000000000000000000000000000000EB
:1055C00000000000000000000000000000000000DB
:1055D00000000000000000000000000000000000CB
:1055E00000000000000000000000000000000000BB
:1055F00000040000696E636F6D696E672200000031
:10560000000000000000000000000000000000009A
:10561000000000000000000000000000000000008A
:10562000000000000000000000000000000000007A
:10563000000000000000000000000000000000006A
:10564000000000000000000000000000000000005A
:10565000000000000000000000080000706470649A
:10566000656163742200000000000000000000007B
:10567000000000000000000000000000000000002A
:10568000000000000000000000000000000000001A
:10569000000000000000000000000000000000000A
:1056A00000000000000000000000000000000000FA
:1056B00000000000000000000000000000000000EA
:1056C000001000002B4D444E534749503A00000053
:1056D00000000000000000000000000000000000CA
:1056E00000000000000000000000000000000000BA
:1056F00000000000000000000000000000000000AA
:105700000000000000000000000000000000000099
:105710000000000000000000000000000000000089
:105720000000000000000000400000004552524F01
:10573000520D0A0000000000000000000000000000
:105740000000000000000000000000000000000059
:105750000000000000000000000000000000000049
:105760000000000000000000000000000000000039
:105770000000000000000000000000000000000029
:105780000000000000000000000000000000000019
:1057900000800000434D45204552524F523A0000D0
:1057A00000000000000000000000000000000000F9
:1057B00000000000000000000000000000000000E9
:1057C00000000000000000000000000000000000D9
:1057D00000000000000000000000000000000000C9
:1057E00000000000000000000000000000000000B9
:1057F0000000000000000000002000004552524F51
:10580000520D0A000000000000000000000000002F
:105810000000000000000000000000000000000088
:105820000000000000000000000000000000000078
:105830000000000000000000000000000000000068
:105840000000000000000000000000000000000058
:105850000000000000000000000000000000000048
:10586000020000004F4B0D0A000000000000000085
:105870000000000000000000000000000000000028
:105880000000000000000000000000000000000018
:105890000000000000000000000000000000000008
:1058A00000000000000000000000000000000000F8
:1058B00000000000000000000000000000000000E8
:1058C0000000000000000000200000004F50454E86
:1058D0003A0000000000000000000000000000008E
:1058E00000000000000000000000000000000000B8
:1058F00000000000000000000000000000000000A8
:105900000000000000000000000000000000000097
:105910000000000000000000000000000000000087
:105920000000000000000000000000000000000077
:105930000400000072656164790D0A000000000037
:105940000000000000000000000000000000000057
:105950000000000000000000000000000000000047
:105960000000000000000000000000000000000037
:105970000000000000000000000000000000000027
:105980000000000000000000000000000000000017
:105990000000000000000000000008000D0A0D0AD1
:1059A0004F4B00000000000000000000000000005D
:1059B00000000000000000000000000000000000E7
:1059C00000000000000000000000000000000000D7
:1059D00000000000000000000000000000000000C7
:1059E00000000000000000000000000000000000B7
:1059F00000000000000000000000000000000000A7
:105A0000100008000D0A0D0A000000000000000050
:105A10000000000000000000000000000000000086
:105A20000000000000000000000000000000000076
:105A30000000000000000000000000000000000066
:105A40000000000000000000000000000000000056
:105A50000000000000000000000000000000000046
:105A60000000000000000000010000000D0A00001E
:105A70000000000000000000000000000000000026
:105A80000000000000000000000000000000000016
:105A90000000000000000000000000000000000006
:105AA00000000000000000000000000000000000F6
:105AB00000000000000000000000000000000000E6
:105AC00000000000000000000000000000000000D6
:105AD0005375636365737366756C20496E69746989
:105AE000616C697A6174696F6E206F662074686595
:105AF000204D6F64756C650D0A0D0A005369676E61
:105B0000616C205175616C697479204C6576656CA7
:105B10002025642064426D202847534D20466F7233
:105B20006D61743A20256C64290D0A005369676E13
:105B3000616C205175616C697479204C6576656C77
:105B4000206E6F742064657465637461626C650DAA
:105B50000A0000000D0A203E3E3E204D6F64756C29
:105B60006520526567697374726174696F6E205342
:105B700075636365737366756C0D0A0D0A0000002A
:105B80000D0A203E3E3E204D6F64756C65205265C7
:105B900067697374726174696F6E20547279696E8B
:105BA000670D0A0D0A0000000D0A203E3E3E204D02
:105BB0006F64756C6520526567697374726174698E
:105BC0006F6E2044656E6965640D0A0D0A00000061
:105BD0000D0A203E3E3E204D6F64756C6520526577
:105BE00067697374726174696F6E204661696C6570
:105BF000640D0A0D0A0000000D0A203E3E3E204DB5
:105C00006F64756C6520415420436F6D6D756E69CE
:105C1000636174696F6E204572726F722077697468
:105C20006820746865204465766963650D0A000024
:105C3000203E3E3E20446576696365206D69676855
:105C40007420626520646973636F6E6E656374654A
:105C500064206F722077726F6E676C7920636F6E4D
:105C60006E65637465640D0A0D0A0000203E3E3EB9
:105C700020506C6561736520636865636B2069669D
:105C8000207468652053494D20697320696E7365DF
:105C90007274656420616E642076616C69642C2086
:105CA00069662063726564656E7469616C732061F6
:105CB0007265206F6B2C206574632E0D0A0D0A002F
:105CC00000002115110E0D0C0B0B0A0A0909090918
:105CD000090808080808080807070707070707074B
:105CE00007070707070000003031323334353637F5
:105CF00038396162636465666768696A6B6C6D6E8A
:105D00006F707172737475767778797A000000001D
:105D100080B50D49794430310C4A7A442E32914293
:105D200003D00B49AFF3008002BD8DF800000122C3
:105D300069460120FDF712F8012802D19DF8000004
:105D400002BD4FF0FF3002BDB8A2FFF7B4A2FFF7CB
:105D50009000002030B4002512E050F8042BD30747
:105D600044BF4A44521E091F042942F8045BFAD278
:105D700013468C0744BF15809B1CC90748BF1D7084
:105D800050F8041B0029E8D130BC7047FEE7FEE75D
:105D9000FEE7FEE7FEE770477047704700F010B877
:105DA00080B580210348FDF7BEFF0348BDE80240EF
:105DB000FBF7F6BF00040242BC09002000F008B85F
:105DC00002494A68087882184A607047000000203B
:105DD0000349C8680A6882430A60486000F002B854
:105DE000001D0C42704700005369676E616C2069AA
:105DF00073206E6F74206B6E6F776E206F72206EE3
:105E00006F742064657465637461626C6520796584
:105E1000742E2E2E200000004661696C20746F20C5
:105E200041542053594E432C20616674657220738F
:105E300065766572616C20617474656D7074730D44
:105E40000A00000010B5074979441831064C7C441B
:105E5000163404E00A68081D114488470146A1422F
:105E6000F8D110BD7400000090000000202D2D2DF1
:105E7000205155454354454C204547393120506FFA
:105E8000776572205570202D2D2D0D0A0000000021
:105E9000202D2D2D205155454354454C2045473943
:105EA00031205368757420446F776E202D2D2D207E
:105EB0000D0A00004EF68851CEF20001086840F449
:105EC00070000860BFF34F8FBFF36F8F4FF001700A
:105ED000E1EE100A704700007DFEFFFF000A00009F
:105EE000D8000020000000003FB1FFFF9C0100002F
:105EF000A80000000000002000F00DF8002801D0EC
:105F0000FFF7A0FFAFF300800020AFF30080FDF7A4
:105F10006BFB00F002F80120704700F001B80000B0
:105F200007463846FBF74CFEFBE7000005480146F4
:105F300003B4684680F30988AFF30080FFF7BAFF27
:105F4000FFF7DAFFA5EDF5FE38B504460D46284605
:105F5000FFF7DEFEA84218BF0024204632BD000035
:105F60000148804701480047A54400082D5F00080C
:105F70000000000001020304FFF7FEBFFFF7FEBFB1
:105F8000FFF7FEBFFFF7FEBFFFF7FEBFFFF7FEBF45
:105F9000FFF7FEBFFFF7FEBFFFF7FEBFFFF7FEBF35
:105FA000FFF7FEBFFFF7FEBFFFF7FEBFFFF7FEBF25
:105FB000FFF7FEBFFFF7FEBFFFF7FEBFFFF7FEBF15
:105FC000FFF7FEBFFFF7FEBFFFF7FEBFFFF7FEBF05
:105FD000FFF7FEBFFFF7FEBFFFF7FEBFFFF7FEBFF5
:105FE000FFF7FEBFFFF7FEBFFFF7FEBFFFF7FEBFE5
:105FF000FFF7FEBFFFF7FEBFFFF7FEBFFFF7FEBFD5
:10600000FFF7FEBFFFF7FEBFFFF7FEBFFFF7FEBFC4
:10601000FFF7FEBFFFF7FEBFFFF7FEBFFFF7FEBFB4
:10602000FFF7FEBFFFF7FEBFFFF7FEBFFFF7FEBFA4
:10603000FFF7FEBFFFF7FEBFFFF7FEBFFFF7FEBF94
:10604000FFF7FEBFFFF7FEBFFFF7FEBFFFF7FEBF84
:10605000FFF7FEBFFFF7FEBFFFF7FEBFFFF7FEBF74
:10606000FFF7FEBFFFF7FEBFFFF7FEBFFFF7FEBF64
:10607000FFF7FEBFFFF7FEBFFFF7FEBFFFF7FEBF54
:10608000FFF7FEBFFFF7FEBF43010001221008F03B
:10609000050724F400CA1300080452FF01E3BA10F4
:1060A0001410010000920C214C1148F30220000151
:1060B0001003811A00087504129504F10320618809
:1060C000100702040101500A0020A00452500421CC
:0C60D0001B610812D460F206C064A1013C
:0400000508005F2D63
:00000001FF
